:10000000050C66003B0C0600050C02009F0C270047
:10001000500C28000A0C2900310C2A0006020B0E95
:10002000A701A9014509AD050D022C00040C2E0005
:10003000610046050400EE02200A040C2E00290986
:100040000C0281014307200A460401024307250AE6
:10005000190A450966072D030D0303073A0A1F0E07
:10006000EC01AC070008CC070008EC070008E00C26
:100070002C0000081F0EAC00AC060008CC060008DF
:10008000EC060008200C2C0000086D00060C2F0068
:100090008A032B004A03AB016B0367036803690300
:0A00A0006A036D03EF02480A00082E
:00000001FF
